:100000000C9467010C948F010C948F010C948F0158
:100010000C948F010C948F010C948F010C948F0120
:100020000C948F010C948F010C9484060C94500551
:100030000C948F010C948F010C948F010C948F0100
:100040000C948F010C948F010C948F010C948F01F0
:100050000C948F010C948F010C948F010C94A901C6
:100060000C948F010C948F010C948F010C948F01D0
:100070000C948F010C948F010C948F010C948F01C0
:100080000C948F010C948F010C948F010C948F01B0
:100090000C948F010C948F010C948F010C948F01A0
:1000A0000C948F010C948F010C948F01AC02AF0261
:1000B0009E02A202A802D002D002D002B302B7026E
:1000C000BB02C102C502D002CB020000000200093F
:1000D0000F0000030401000C0000000000000000FD
:1000E00000000000000000000408020110408040F1
:1000F000102040804080080204018040201002014E
:10010000108010204040040404040403040502028B
:1001100002020403020202020606060606060404A0
:100120000202020400000000250028002B002E001F
:10013000310000000000240027002A002D003000BC
:1001400000C18081C112010002020000404123363B
:100150008000010102000112010002000000404184
:1001600023368000010102000141726475696E6FDF
:10017000204C4C430041726475696E6F204C656F72
:100180006E6172646F0004030904080B000202022E
:100190000100090400000102020000052400100112
:1001A00005240101010424020605240600010705B7
:1001B000810310004009040100020A000000070545
:1001C000020240000007058302400000000000001A
:1001D000000000002A2B28000000000000000000A2
:1001E0000000000000000000000000002C9EB4A0F1
:1001F000A1A2A434A6A7A5AE362D3738271E1F20EE
:10020000212223242526B333B62EB7B89F848586B2
:100210008788898A8B8C8D8E8F90919293949596F6
:100220009798999A9B9C9D2F3130A3AD3504050674
:100230000708090A0B0C0D0E0F10111213141516D6
:100240001718191A1B1C1DAFB1B0B5000904020024
:1002500001030000000921010100012265000705DA
:10026000840340000105010902A1010901A10085E3
:10027000010509190129031500250195037501815F
:100280000295017505810305010930093109381509
:1002900081257F750895038106C0C005010906A167
:1002A000018502050719E029E7150025017501956B
:1002B00008810295017508810395067508150025CA
:1002C000650507190029658100C0B60709091124D1
:1002D0001FBECFEFDAE0DEBFCDBF11E0A0E0B1E09E
:1002E000ECE8F2E102C005900D92A832B107D9F70F
:1002F00021E0A8E2B1E001C01D92A739B207E1F701
:1003000012E0CEECD2E004C02297FE010E94400928
:10031000CA3CD107C9F70E9441030C9444090C94CC
:10032000000061E08DE00C94D10261E08DE00E945C
:100330000A0368EE73E080E090E00E94160260E03D
:100340008DE00E940A0368EE73E080E090E00C9478
:1003500016021F920F920FB60F9211242F933F9304
:100360008F939F93AF93BF938091290190912A011E
:10037000A0912B01B0912C013091280123E0230F93
:100380002D3720F40196A11DB11D05C026E8230FCD
:100390000296A11DB11D20932801809329019093FD
:1003A0002A01A0932B01B0932C0180912D019091F3
:1003B0002E01A0912F01B09130010196A11DB11D18
:1003C00080932D0190932E01A0932F01B0933001C3
:1003D000BF91AF919F918F913F912F910F900FBE41
:1003E0000F901F9018953FB7F89480912D01909130
:1003F0002E01A0912F01B091300126B5A89B05C018
:100400002F3F19F00196A11DB11D3FBF6627782F20
:10041000892F9A2F620F711D811D911D42E0660F79
:10042000771F881F991F4A95D1F70895CF92DF92C1
:10043000EF92FF92CF93DF936B017C010E94F30157
:10044000EB01C114D104E104F10489F00E94F80623
:100450000E94F3016C1B7D0B683E734090F381E0BA
:10046000C81AD108E108F108C851DC4FEACFDF9182
:10047000CF91FF90EF90DF90CF900895789484B55E
:10048000826084BD84B5816084BD85B5826085BD90
:1004900085B5816085BDEEE6F0E080818160808376
:1004A000E1E8F0E010828081826080838081816059
:1004B0008083E0E8F0E0808181608083E1E9F0E022
:1004C000808182608083808181608083E0E9F0E0C8
:1004D000808181608083E1ECF0E0808184608083B2
:1004E000808182608083808181608083E3ECF0E0A2
:1004F000808181608083E0ECF0E080818260808395
:10050000E2ECF0E0808181608083EAE7F0E08081C6
:100510008460808380818260808380818160808329
:10052000808180688083089590E0FC013197EF30EE
:10053000F105B0F5EA5AFF4F0C943E098091800016
:100540008F7703C0809180008F7D80938000089515
:1005500080918000877FF9CF84B58F7702C084B502
:100560008F7D84BD0895809190008F7707C0809122
:1005700090008F7D03C080919000877F80939000D2
:1005800008958091C0008F7703C08091C0008F7D57
:100590008093C00008958091C200877F8093C2003D
:1005A0000895CF93DF9390E0FC01E851FF4F249131
:1005B000FC01EA5FFE4F8491882349F190E0880FA7
:1005C000991FFC01EE5CFE4FA591B4918C5D9E4F8E
:1005D000FC01C591D4919FB7611108C0F8948C912A
:1005E000209582238C93888182230AC0623051F443
:1005F000F8948C91322F309583238C938881822BB1
:10060000888304C0F8948C91822B8C939FBFDF91D8
:10061000CF9108950F931F93CF93DF931F92CDB780
:10062000DEB7282F30E0F901E653FF4F8491F9013E
:10063000E851FF4F1491F901EA5FFE4F0491002346
:10064000C9F0882321F069830E9494026981E02F18
:10065000F0E0EE0FFF1FEC5DFE4FA591B4919FB748
:10066000F8948C91611103C01095812301C0812BF6
:100670008C939FBF0F90DF91CF911F910F910895A1
:1006800008950E943E020E94400381E391E00E948F
:10069000DA060E949101C0E0D0E00E949501209707
:1006A000E1F30E940000F9CF4091350150913601ED
:1006B000209133013091340142175307B4F49091E3
:1006C000E8009570E1F39091E80092FD19C08093E5
:1006D000F100809135019091360101968F73992731
:1006E000892B19F48EEF8093E80080913501909169
:1006F00036010196909336018093350181E008958B
:1007000080E00895CF92DF92FF920F931F93CF93D3
:10071000DF931F92CDB7DEB7082F162F862F880FD5
:100720008E5F99830E94540383E00E945403F02E4D
:10073000C02E9981D92E8C2D8F19811778F4F6014E
:1007400084910E945403082F80E00E945403802368
:10075000FFEFCF1ADF0A8111EECF01C081E00F90C9
:10076000DF91CF911F910F91FF90DF90CF9008956F
:10077000615030F02091F100FC0120830196F8CF08
:10078000289884E68093380108952FB7FC012083D0
:10079000F89467706093E9000895CF93DF931F92F8
:1007A000CDB7DEB7682FCE0101960E94C5038091B8
:1007B000F20099819FBF0F90DF91CF910895FF9232
:1007C0000F931F93CF93DF9300D0CDB7DEB7F62EF4
:1007D0008A0190913701992311F057FF03C08FEFE1
:1007E0009FEF2BC0682FCE0101967A830E94C5032C
:1007F0008091F20090E0A8017A81801791070CF4B3
:10080000AC01EF2DF72FF40E84E6FE1639F0289890
:10081000809338019091F1009193F7CF41155105E4
:1008200021F08091F200882321F089818FBFCA01D5
:1008300004C08BE68093E800F8CF0F900F90DF9113
:10084000CF911F910F91FF900895CF93DF931F9247
:10085000CDB7DEB741E050E0BE016F5F7F4F0E9431
:10086000DF03019719F4898190E002C08FEF9FEFB9
:100870000F90DF91CF910895CF93DF931F92CDB763
:10088000DEB7682FCE0101960E94C5039091E80063
:10089000892F807295FF04C09091F20080E4891B3B
:1008A00099819FBF0F90DF91CF9108956F927F92B2
:1008B0008F929F92AF92BF92CF92DF92EF92FF9270
:1008C0000F931F93CF93DF931F92CDB7DEB7782E90
:1008D0007B01C42EB52E80913701882369F0042F47
:1008E000152F8AEFD82E872D8072982E9AE3A92E85
:1008F000872D8074882E11C08FEF9FEF57C0872DF2
:100900000E943C04682E81110CC0DA94A9F361E0C6
:1009100070E080E090E00E9416020115110579F761
:100920003BC0282F30E0021713070CF4602E672D10
:10093000CE0101960E94C5038091E80085FF29C081
:10094000262D30E0021B130B992039F06A948FEFAB
:100950006816B1F01092F100F9CFF701862D77FEFD
:1009600007C0815058F094919093F1003196F9CFDF
:10097000815020F091919093F100FACFE20EF31E96
:100980008091E80085FF0FC00115110511F4811059
:100990000AC089818FBFC1CF5D9884E680933901F9
:1009A0008C2D9B2D03C0A092E800F3CF0F90DF9118
:1009B000CF911F910F91FF90EF90DF90CF90BF905C
:1009C000AF909F908F907F906F9008951092E90064
:1009D00010923601109235019093340180933301C7
:1009E0000895CF92DF92FF920F931F93CF93DF93DF
:1009F00000D0CDB7DEB7F82E8A016B0101151105C5
:100A0000B1F0F601F7FE02C0849101C080814983F4
:100A10005A830E94540301501109FFEFCF1ADF0AD5
:100A200049815A818111EACF8FEF9FEF01C0CA013E
:100A30000F900F90DF91CF911F910F91FF90DF905A
:100A4000CF9008951F93CF93DF931F92CDB7DEB75A
:100A5000162F2091E80022FFFCCF612F79830E949E
:100A6000B8038BEF8093E800812F7981972F0F9047
:100A7000DF91CF911F910895CF93DF931F92CDB750
:100A8000DEB71982CE0101960E945607CE0101966B
:100A90000E94F107898190E00F90DF91CF91089536
:100AA0001F920F920FB60F921124EF92FF920F93A5
:100AB0001F932F933F934F935F936F937F938F93E6
:100AC0009F93AF93BF93EF93FF93CF93DF93CDB7F4
:100AD000DEB76297DEBFCDBF1092E9008091E800DB
:100AE00083FFEBC068E0CE010A960E94B80382EF54
:100AF0008093E8009A8597FF05C08091E80080FF09
:100B0000FCCF03C08EEF8093E800892F807609F038
:100B1000B9C08B85811105C01092F1001092F100CF
:100B2000C5C0282F2D7F213009F4C0C0853049F47D
:100B30008091E80080FFFCCF8C8580688093E30083
:100B4000B5C0863009F076C02D85E888F988223056
:100B500071F580E090E02A8B0E94E6040E943C053B
:100B600099E08E010F5F1F4FF801392F11923A95CE
:100B7000E9F799832A892A8391E09E8390E89887F0
:100B80009AEF99872091350130913601275F3F4FC9
:100B90003C832B838D83C7010E94E60449E050E02B
:100BA000B80180E00E94F1040E943C057FC0C701AB
:100BB0002A8B0E94E6042A89223241F482E290E0E4
:100BC0000E94FC07892B09F071C074C0213069F4C0
:100BD00088899989089711F4209332018091320114
:100BE000811118C067E571E01AC0233009F062C0B6
:100BF0008C85882391F0823021F460E185E791E0D3
:100C000006C0813009F056C06BE089E691E00E9491
:100C100082034AC065E471E002C066E871E06115D4
:100C2000710509F447C0FB01449150E080E80E943F
:100C3000F1043CC0873009F43DC0883021F481E0E4
:100C40008093F10033C0893089F5937099F5E1E420
:100C5000F1E081E021E096E38093E9002093EB004E
:100C600034913093EC009093ED008F5F3196853096
:100C700099F78EE78093EA001092EA008C858093C2
:100C8000370114C0888999890E94E6048E858111F4
:100C900005C0CE010A960E94610706C0823051F459
:100CA000CE010A960E942408882321F08EEF8093BB
:100CB000E80003C081E28093EB0062960FB6F894DF
:100CC000DEBF0FBECDBFDF91CF91FF91EF91BF91FE
:100CD000AF919F918F917F916F915F914F913F91D4
:100CE0002F911F910F91FF90EF900F900FBE0F90DB
:100CF0001F9018958093E9008091F200882319F0E5
:100D00008AE38093E80008951F920F920FB60F9226
:100D100011242F933F934F935F936F937F938F9300
:100D20009F93AF93BF93EF93FF938091E100109255
:100D3000E10083FF0FC01092E90091E09093EB0077
:100D40001092EC0092E39093ED001092370198E03E
:100D50009093F00082FF1DC083E00E947A0680918C
:100D60003901882339F0809139018150809339010C
:100D7000882369F080913801882359F080913801E7
:100D8000815080933801811104C0289A02C05D9A75
:100D9000F1CFFF91EF91BF91AF919F918F917F9193
:100DA0006F915F914F913F912F910F900FBE0F90D8
:100DB0001F9018951092370181E08093D70080EA48
:100DC0008093D80082E189BD09B400FEFDCF61E0C7
:100DD00070E080E090E00E94160280E98093D800E5
:100DE0008CE08093E2001092E000559A209A0895DA
:100DF0000895CF93DF931F92CDB7DEB76983DC01EF
:100E0000ED91FC910280F381E02D41E050E0BE01C4
:100E10006F5F7F4F09950F90DF91CF910895CF932A
:100E2000DF93EC018C859D8597FF05C082E00E94D1
:100E300025049D878C878C859D85DF91CF910895B2
:100E400083E00C947A06FC018485958597FD06C0A5
:100E500082E00E94CD0390E00196089582E00E9416
:100E6000CD0390E00895FC018485958597FD05C02C
:100E70002FEF3FEF35872487089582E00C942504F7
:100E8000CF93DF93EC0180910701882331F083E059
:100E90000E9456041816190634F081E090E09B83F6
:100EA0008A8380E090E0DF91CF910895FC0120815A
:100EB0002E5F208342E450E06AE871E080E80C9401
:100EC000F104FC0181819081913A59F4813209F059
:100ED0003CC047E050E060E071E080E00E94F10437
:100EE00043C0913291F5803239F467E070E080E0E0
:100EF00091E00E94220506C0823209F035C082814D
:100F0000809307018091000190910101A09102015D
:100F1000B0910301803B9440A105B105C1F48091DB
:100F2000070180FD14C087E797E79093010880933D
:100F300000082BE088E190E00FB6F894A895809324
:100F400060000FBE209360000FC080E0089588E12C
:100F50000FB6F89480936000109260000FBEA895C1
:100F6000109201081092000881E0089510923D014E
:100F700010923C0188EE93E0A0E0B0E080933E0147
:100F800090933F01A0934001B09341018EE091E026
:100F900090933B0180933A018FEF9FEF909347012D
:100FA000809346010895FF920F931F93CF93DF9391
:100FB000EC01F62EE881F9810480F581E02D099598
:100FC0008C01E881F9810680F781E02D6F2DCE013B
:100FD0000995C8019927DF91CF911F910F91FF903B
:100FE0000895FC0120812F5F208349E150E06CE4EB
:100FF00072E080E80C94F10445E650E065E672E0AA
:1010000080E80C94F104EF92FF920F931F93CF931B
:10101000DF931F92CDB7DEB789838B017A0141E060
:1010200050E0BE016F5F7F4F84E00E945604A7012D
:10103000B80184E40E9456040F90DF91CF911F9174
:101040000F91FF90EF900895FC0191818081813A8A
:1010500031F481E0913091F0933089F411C0813204
:1010600071F49B3021F482818093090105C09A308C
:1010700031F482818093080181E00895089580E031
:10108000089548E050E082E00C940308CF93DF938A
:10109000DC01683818F0E8E7E60F25C0E62FF0E03D
:1010A00067FF11C0E058F10981E090E001C0880FAE
:1010B000EA95EAF714969C911497982B14969C93B2
:1010C0001497E0E010C0E453FE4FE491EE2309F4DE
:1010D00040C0E7FF08C014968C9114978260149664
:1010E0008C931497EF7716968C9116978E1741F183
:1010F00017968C9117978E1719F118968C9118974F
:101100008E17F1F019968C9119978E17C9F01A96CF
:101110008C911A978E17A1F01B968C911B978E17A6
:1011200079F080E090E0ED01C80FD91F2E812111E8
:1011300002C0EE8305C0019686309105A1F709C073
:10114000BD016C5F7F4FCD010E94410881E090E0BE
:1011500008C081E090E013969C938E93129780E0F4
:1011600090E0DF91CF910895683818F0E8E7E60F36
:1011700025C0E62FF0E067FF12C0E058F10921E03A
:1011800030E001C0220FEA95EAF72095DC011496C1
:101190003C911497322314963C93E0E00FC0E45343
:1011A000FE4FE491EE2329F1E7FF08C0DC0114961D
:1011B0002C9114972D7F14962C93EF7720E030E03C
:1011C000EE2351F0DC01A20FB31F16964C91169737
:1011D0004E1302C016961C922F5F3F4F26303105EA
:1011E00079F7BC016C5F7F4F0E94410881E090E07D
:1011F000089580E090E00895FC0116821782108621
:101200001186128613861482BC016C5F7F4F0C948A
:1012100041081092960110928D0110928C018EE17E
:1012200091E090938B0180938A010895CF92DF9291
:10123000EF92FF920F931F93CF93DF936C017A018C
:10124000EB01E60EF71E00E010E0CE15DF0561F0C1
:101250006991D601ED91FC910190F081E02DC601DC
:101260000995080F191FF1CFC801DF91CF911F9188
:101270000F91FF90EF90DF90CF900895EE0FFF1F3A
:0C1280000590F491E02D0994F894FFCF44
:10128C0000E1000000000000010100000000F90670
:10129C004007230733070F07200700000000D30780
:0812AC0016094608B408FC080D
:00000001FF
